 saproc

 Timestamp is 2c652a83 (reproducible build file hash)

 Preferred load address is 10000000

 Start         Length     Name                   Class
 0001:00000000 00002d2fH .text$mn                CODE
 0001:00002d2f 000001d8H .text$x                 CODE
 0002:00000000 000000e0H .idata$5                DATA
 0002:000000e0 00000008H .00cfg                  DATA
 0002:000000e8 00000004H .CRT$XCA                DATA
 0002:000000ec 00000004H .CRT$XCZ                DATA
 0002:000000f0 00000004H .CRT$XIA                DATA
 0002:000000f4 00000004H .CRT$XIZ                DATA
 0002:000000f8 00000004H .CRT$XPA                DATA
 0002:000000fc 00000004H .CRT$XPZ                DATA
 0002:00000100 00000004H .CRT$XTA                DATA
 0002:00000104 00000004H .CRT$XTZ                DATA
 0002:00000108 00000000H .gfids$y                DATA
 0002:00000108 00000978H .rdata                  DATA
 0002:00000a80 00000000H .rdata$CastGuardVftablesA DATA
 0002:00000a80 00000000H .rdata$CastGuardVftablesC DATA
 0002:00000a80 000001e8H .rdata$r                DATA
 0002:00000c68 00000024H .rdata$sxdata           DATA
 0002:00000c8c 0000006cH .rdata$voltmd           DATA
 0002:00000cf8 000002e4H .rdata$zzzdbg           DATA
 0002:00000fdc 00000004H .rtc$IAA                DATA
 0002:00000fe0 00000004H .rtc$IZZ                DATA
 0002:00000fe4 00000004H .rtc$TAA                DATA
 0002:00000fe8 00000008H .rtc$TZZ                DATA
 0002:00000ff0 00000340H .xdata$x                DATA
 0002:00001330 000003dcH .edata                  DATA
 0002:0000170c 000000a0H .idata$2                DATA
 0002:000017ac 00000014H .idata$3                DATA
 0002:000017c0 000000e0H .idata$4                DATA
 0002:000018a0 0000046eH .idata$6                DATA
 0003:00000000 00000018H .data                   DATA
 0003:00000018 00000060H .data$r                 DATA
 0003:00000078 00000078H .data$rs                DATA
 0003:000000f0 000003a4H .bss                    DATA
 0004:00000000 00000060H .rsrc$01                DATA
 0004:00000060 00000328H .rsrc$02                DATA

  Address         Publics by Value              Rva+Base       Lib:Object

 0000:00000000       ___AbsoluteZero            00000000     <absolute>
 0000:00000000       ___arm64x_extra_rfe_table  00000000     <absolute>
 0000:00000000       ___arm64x_extra_rfe_table_size 00000000     <absolute>
 0000:00000000       ___arm64x_native_entrypoint 00000000     <absolute>
 0000:00000000       ___arm64x_redirection_metadata 00000000     <absolute>
 0000:00000000       ___arm64x_redirection_metadata_count 00000000     <absolute>
 0000:00000000       ___dynamic_value_reloc_table 00000000     <absolute>
 0000:00000000       ___enclave_config          00000000     <absolute>
 0000:00000000       ___guard_check_icall_a64n_fptr 00000000     <absolute>
 0000:00000000       ___guard_eh_cont_count     00000000     <absolute>
 0000:00000000       ___guard_eh_cont_table     00000000     <absolute>
 0000:00000000       ___guard_fids_count        00000000     <absolute>
 0000:00000000       ___guard_fids_table        00000000     <absolute>
 0000:00000000       ___guard_iat_count         00000000     <absolute>
 0000:00000000       ___guard_iat_table         00000000     <absolute>
 0000:00000000       ___guard_longjmp_count     00000000     <absolute>
 0000:00000000       ___guard_longjmp_table     00000000     <absolute>
 0000:00000000       ___hybrid_auxiliary_delayload_iat 00000000     <absolute>
 0000:00000000       ___hybrid_auxiliary_delayload_iat_copy 00000000     <absolute>
 0000:00000000       ___hybrid_auxiliary_iat    00000000     <absolute>
 0000:00000000       ___hybrid_auxiliary_iat_copy 00000000     <absolute>
 0000:00000000       ___hybrid_code_map         00000000     <absolute>
 0000:00000000       ___hybrid_code_map_count   00000000     <absolute>
 0000:00000000       ___hybrid_image_info_bitfield 00000000     <absolute>
 0000:00000000       ___x64_code_ranges_to_entry_points 00000000     <absolute>
 0000:00000000       ___x64_code_ranges_to_entry_points_count 00000000     <absolute>
 0000:00000009       ___safe_se_handler_count   00000009     <absolute>
 0000:00000100       ___guard_flags             00000100     <absolute>
 0000:00000000       ___ImageBase               10000000     <linker-defined>
 0001:00000000       _Java_sun_jvm_hotspot_asm_Disassembler_decode@36 10001000 f   sadis.obj
 0001:00000186       _Java_sun_jvm_hotspot_asm_Disassembler_load_1library@12 10001186 f   sadis.obj
 0001:0000025e       ___local_stdio_printf_options 1000125e f i sadis.obj
 0001:00000264       __vsnprintf_l              10001264 f i sadis.obj
 0001:0000049e       ??_GSAOutputCallbacks@@QAEPAXI@Z 1000149e f i sawindbg.obj
 0001:000004c3       ?AddRef@SAOutputCallbacks@@UAGKXZ 100014c3 f   sawindbg.obj
 0001:000004d3       ?CallObjectMethod@JNIEnv_@@QAAPAV_jobject@@PAV2@PAU_jmethodID@@ZZ 100014d3 f i sawindbg.obj
 0001:000004ee       ?CallVoidMethod@JNIEnv_@@QAAXPAV_jobject@@PAU_jmethodID@@ZZ 100014ee f i sawindbg.obj
 0001:00000509       ?Output@SAOutputCallbacks@@UAGJKPBD@Z 10001509 f   sawindbg.obj
 0001:00000586       ?QueryInterface@SAOutputCallbacks@@UAGJABU_GUID@@PAPAX@Z 10001586 f   sawindbg.obj
 0001:000005d5       ?Release@SAOutputCallbacks@@UAGKXZ 100015d5 f   sawindbg.obj
 0001:000005f6       ?SetLongField@JNIEnv_@@QAEXPAV_jobject@@PAU_jfieldID@@_J@Z 100015f6 f i sawindbg.obj
 0001:00000eca       ?clearBuffer@SAOutputCallbacks@@QAEXXZ 10001eca f i sawindbg.obj
 0001:0000156c       _Java_sun_jvm_hotspot_debugger_windbg_WindbgDebuggerLocal_attach0__I@12 1000256c f   sawindbg.obj
 0001:000015b7       _Java_sun_jvm_hotspot_debugger_windbg_WindbgDebuggerLocal_attach0__Ljava_lang_String_2Ljava_lang_String_2@16 100025b7 f   sawindbg.obj
 0001:00001602       _Java_sun_jvm_hotspot_debugger_windbg_WindbgDebuggerLocal_consoleExecuteCommand0@12 10002602 f   sawindbg.obj
 0001:0000183c       _Java_sun_jvm_hotspot_debugger_windbg_WindbgDebuggerLocal_detach0@8 1000283c f   sawindbg.obj
 0001:00001878       _Java_sun_jvm_hotspot_debugger_windbg_WindbgDebuggerLocal_getThreadIdFromSysId0@16 10002878 f   sawindbg.obj
 0001:000018dd       _Java_sun_jvm_hotspot_debugger_windbg_WindbgDebuggerLocal_initIDs@8 100028dd f   sawindbg.obj
 0001:00001abb       _Java_sun_jvm_hotspot_debugger_windbg_WindbgDebuggerLocal_lookupByAddress0@16 10002abb f   sawindbg.obj
 0001:00001ba6       _Java_sun_jvm_hotspot_debugger_windbg_WindbgDebuggerLocal_lookupByName0@16 10002ba6 f   sawindbg.obj
 0001:00001c63       _Java_sun_jvm_hotspot_debugger_windbg_WindbgDebuggerLocal_readBytesFromProcess0@24 10002c63 f   sawindbg.obj
 0001:00001d21       __vfprintf_l               10002d21 f i sawindbg.obj
 0001:00001d45       _fprintf                   10002d45 f i sawindbg.obj
 0001:00001d5d       _printf                    10002d5d f i sawindbg.obj
 0001:00001d7b       _snprintf                  10002d7b f i sawindbg.obj
 0001:00001d95       _vsnprintf                 10002d95 f i sawindbg.obj
 0001:00001dc7       _DebugCreate@8             10002dc7 f   dbgeng:dbgeng.dll
 0001:00001dcd       _JNU_NewStringPlatform@8   10002dcd f   java:java.dll
 0001:00001dd3       _JNU_NewObjectByName       10002dd3 f   java:java.dll
 0001:00001dd9       _getLastErrorString@8      10002dd9 f   java:java.dll
 0001:00001ddf       @__security_check_cookie@4 10002ddf f   MSVCRT:secchk.obj
 0001:00001df0       __alloca_probe             10002df0 f   MSVCRT:chkstk.obj
 0001:00001df0       __chkstk                   10002df0 f   MSVCRT:chkstk.obj
 0001:00001e1b       ??2@YAPAXI@Z               10002e1b f   MSVCRT:new_scalar.obj
 0001:00001e4b       ??3@YAXPAXI@Z              10002e4b f   MSVCRT:delete_scalar_size.obj
 0001:00001e59       ??_U@YAPAXI@Z              10002e59 f   MSVCRT:new_array.obj
 0001:00001e62       ??_V@YAXPAX@Z              10002e62 f   MSVCRT:delete_array.obj
 0001:00001e67       __EH_epilog3               10002e67 f   MSVCRT:ehprolg3.obj
 0001:00001e7b       __EH_prolog3               10002e7b f   MSVCRT:ehprolg3.obj
 0001:00001eae       ??_Etype_info@@UAEPAXI@Z   10002eae f i MSVCRT:std_type_info_static.obj
 0001:00001eae       ??_Gtype_info@@UAEPAXI@Z   10002eae f i MSVCRT:std_type_info_static.obj
 0001:00002211       __DllMainCRTStartup@12     10003211 f   MSVCRT:dll_dllmain.obj
 0001:00002234       ___raise_securityfailure   10003234 f   MSVCRT:gs_report.obj
 0001:0000225c       ___report_gsfailure        1000325c f   MSVCRT:gs_report.obj
 0001:00002356       ??0bad_alloc@std@@QAE@ABV01@@Z 10003356 f i MSVCRT:throw_bad_alloc.obj
 0001:00002371       ??0bad_alloc@std@@QAE@XZ   10003371 f i MSVCRT:throw_bad_alloc.obj
 0001:00002389       ??0bad_array_new_length@std@@QAE@ABV01@@Z 10003389 f i MSVCRT:throw_bad_alloc.obj
 0001:000023a4       ??0bad_array_new_length@std@@QAE@XZ 100033a4 f i MSVCRT:throw_bad_alloc.obj
 0001:000023bc       ??0exception@std@@QAE@ABV01@@Z 100033bc f i MSVCRT:throw_bad_alloc.obj
 0001:000023e8       ??1bad_alloc@std@@UAE@XZ   100033e8 f i MSVCRT:throw_bad_alloc.obj
 0001:000023e8       ??1bad_array_new_length@std@@UAE@XZ 100033e8 f i MSVCRT:throw_bad_alloc.obj
 0001:000023f9       ??_Ebad_alloc@std@@UAEPAXI@Z 100033f9 f i MSVCRT:throw_bad_alloc.obj
 0001:000023f9       ??_Ebad_array_new_length@std@@UAEPAXI@Z 100033f9 f i MSVCRT:throw_bad_alloc.obj
 0001:000023f9       ??_Eexception@std@@UAEPAXI@Z 100033f9 f i MSVCRT:throw_bad_alloc.obj
 0001:000023f9       ??_Gbad_alloc@std@@UAEPAXI@Z 100033f9 f i MSVCRT:throw_bad_alloc.obj
 0001:000023f9       ??_Gbad_array_new_length@std@@UAEPAXI@Z 100033f9 f i MSVCRT:throw_bad_alloc.obj
 0001:000023f9       ??_Gexception@std@@UAEPAXI@Z 100033f9 f i MSVCRT:throw_bad_alloc.obj
 0001:00002426       ?__scrt_throw_std_bad_alloc@@YAXXZ 10003426 f   MSVCRT:throw_bad_alloc.obj
 0001:00002443       ?__scrt_throw_std_bad_array_new_length@@YAXXZ 10003443 f   MSVCRT:throw_bad_alloc.obj
 0001:00002460       ?what@exception@std@@UBEPBDXZ 10003460 f i MSVCRT:throw_bad_alloc.obj
 0001:0000246d       ??3@YAXPAX@Z               1000346d f   MSVCRT:delete_scalar.obj
 0001:000024bf       ___security_init_cookie    100034bf f   MSVCRT:gs_support.obj
 0001:0000250a       _DllMain@12                1000350a f   MSVCRT:dll_dllmain_stub.obj
 0001:0000252c       ?__scrt_initialize_type_info@@YAXXZ 1000352c f   MSVCRT:tncleanup.obj
 0001:00002538       ?__scrt_uninitialize_type_info@@YAXXZ 10003538 f   MSVCRT:tncleanup.obj
 0001:00002544       ___local_stdio_scanf_options 10003544 f i MSVCRT:default_local_stdio_options.obj
 0001:0000254a       ___scrt_initialize_default_local_stdio_options 1000354a f   MSVCRT:default_local_stdio_options.obj
 0001:000025ab       ___scrt_acquire_startup_lock 100035ab f   MSVCRT:utility.obj
 0001:000025dd       ___scrt_dllmain_after_initialize_c 100035dd f   MSVCRT:utility.obj
 0001:00002608       ___scrt_dllmain_before_initialize_c 10003608 f   MSVCRT:utility.obj
 0001:00002616       ___scrt_dllmain_crt_thread_attach 10003616 f   MSVCRT:utility.obj
 0001:00002635       ___scrt_dllmain_crt_thread_detach 10003635 f   MSVCRT:utility.obj
 0001:00002642       ___scrt_dllmain_exception_filter 10003642 f   MSVCRT:utility.obj
 0001:00002676       ___scrt_dllmain_uninitialize_c 10003676 f   MSVCRT:utility.obj
 0001:00002699       ___scrt_dllmain_uninitialize_critical 10003699 f   MSVCRT:utility.obj
 0001:000026a6       ___scrt_initialize_crt     100036a6 f   MSVCRT:utility.obj
 0001:000026df       ___scrt_initialize_onexit_tables 100036df f   MSVCRT:utility.obj
 0001:00002766       ___scrt_is_nonwritable_in_current_image 10003766 f   MSVCRT:utility.obj
 0001:000027fa       ___scrt_release_startup_lock 100037fa f   MSVCRT:utility.obj
 0001:00002817       ___scrt_uninitialize_crt   10003817 f   MSVCRT:utility.obj
 0001:0000283f       ___scrt_get_dyn_tls_init_callback 1000383f f   MSVCRT:dyn_tls_init.obj
 0001:00002845       ___scrt_fastfail           10003845 f   MSVCRT:utility_desktop.obj
 0001:00002960       __crt_debugger_hook        10003960 f   MSVCRT:utility_desktop.obj
 0001:00002968       __RTC_Initialize           10003968 f   MSVCRT:initsect.obj
 0001:00002994       __RTC_Terminate            10003994 f   MSVCRT:initsect.obj
 0001:000029c0       __SEH_prolog4              100039c0 f   MSVCRT:sehprolg4.obj
 0001:00002a05       __except_handler4          10003a05 f   MSVCRT:chandler4gs.obj
 0001:00002a34       @_guard_check_icall_nop@4  10003a34 f i MSVCRT:guard_support.obj
 0001:00002a37       ___isa_available_init      10003a37 f   MSVCRT:cpu_disp.obj
 0001:00002c0b       __get_startup_argv_mode    10003c0b f   MSVCRT:argv_mode.obj
 0001:00002c0f       ___scrt_is_ucrt_dll_in_use 10003c0f f   MSVCRT:ucrt_detection.obj
 0001:00002c1b       _strchr                    10003c1b f   vcruntime:VCRUNTIME140.dll
 0001:00002c21       ___std_terminate           10003c21 f   vcruntime:VCRUNTIME140.dll
 0001:00002c27       _memcmp                    10003c27 f   vcruntime:VCRUNTIME140.dll
 0001:00002c2d       _memset                    10003c2d f   vcruntime:VCRUNTIME140.dll
 0001:00002c33       _strstr                    10003c33 f   vcruntime:VCRUNTIME140.dll
 0001:00002c39       ___CxxFrameHandler3        10003c39 f   vcruntime:VCRUNTIME140.dll
 0001:00002c3f       ___std_exception_copy      10003c3f f   vcruntime:VCRUNTIME140.dll
 0001:00002c45       ___std_exception_destroy   10003c45 f   vcruntime:VCRUNTIME140.dll
 0001:00002c4b       __CxxThrowException@8      10003c4b f   vcruntime:VCRUNTIME140.dll
 0001:00002c51       ___std_type_info_destroy_list 10003c51 f   vcruntime:VCRUNTIME140.dll
 0001:00002c57       __except_handler4_common   10003c57 f   vcruntime:VCRUNTIME140.dll
 0001:00002c5d       _strlen                    10003c5d f   ucrt:api-ms-win-crt-string-l1-1-0.dll
 0001:00002c63       _strcat                    10003c63 f   ucrt:api-ms-win-crt-string-l1-1-0.dll
 0001:00002c69       _strcpy                    10003c69 f   ucrt:api-ms-win-crt-string-l1-1-0.dll
 0001:00002c6f       _free                      10003c6f f   ucrt:api-ms-win-crt-heap-l1-1-0.dll
 0001:00002c75       _malloc                    10003c75 f   ucrt:api-ms-win-crt-heap-l1-1-0.dll
 0001:00002c7b       __callnewh                 10003c7b f   ucrt:api-ms-win-crt-heap-l1-1-0.dll
 0001:00002c81       __initterm                 10003c81 f   ucrt:api-ms-win-crt-runtime-l1-1-0.dll
 0001:00002c87       __initterm_e               10003c87 f   ucrt:api-ms-win-crt-runtime-l1-1-0.dll
 0001:00002c8d       __seh_filter_dll           10003c8d f   ucrt:api-ms-win-crt-runtime-l1-1-0.dll
 0001:00002c93       __configure_narrow_argv    10003c93 f   ucrt:api-ms-win-crt-runtime-l1-1-0.dll
 0001:00002c99       __initialize_narrow_environment 10003c99 f   ucrt:api-ms-win-crt-runtime-l1-1-0.dll
 0001:00002c9f       __initialize_onexit_table  10003c9f f   ucrt:api-ms-win-crt-runtime-l1-1-0.dll
 0001:00002ca5       __execute_onexit_table     10003ca5 f   ucrt:api-ms-win-crt-runtime-l1-1-0.dll
 0001:00002cab       __cexit                    10003cab f   ucrt:api-ms-win-crt-runtime-l1-1-0.dll
 0001:00002cb1       ___acrt_initialize         10003cb1 f   MSVCRT:ucrt_stubs.obj
 0001:00002cb1       ___acrt_thread_attach      10003cb1 f   MSVCRT:ucrt_stubs.obj
 0001:00002cb1       ___acrt_thread_detach      10003cb1 f   MSVCRT:ucrt_stubs.obj
 0001:00002cb1       ___acrt_uninitialize       10003cb1 f   MSVCRT:ucrt_stubs.obj
 0001:00002cb1       ___acrt_uninitialize_critical 10003cb1 f   MSVCRT:ucrt_stubs.obj
 0001:00002cb1       ___scrt_stub_for_acrt_initialize 10003cb1 f   MSVCRT:ucrt_stubs.obj
 0001:00002cb1       ___scrt_stub_for_acrt_thread_attach 10003cb1 f   MSVCRT:ucrt_stubs.obj
 0001:00002cb1       ___scrt_stub_for_acrt_thread_detach 10003cb1 f   MSVCRT:ucrt_stubs.obj
 0001:00002cb1       ___scrt_stub_for_acrt_uninitialize 10003cb1 f   MSVCRT:ucrt_stubs.obj
 0001:00002cb1       ___scrt_stub_for_acrt_uninitialize_critical 10003cb1 f   MSVCRT:ucrt_stubs.obj
 0001:00002cb1       ___vcrt_initialize         10003cb1 f   MSVCRT:ucrt_stubs.obj
 0001:00002cb1       ___vcrt_thread_attach      10003cb1 f   MSVCRT:ucrt_stubs.obj
 0001:00002cb1       ___vcrt_thread_detach      10003cb1 f   MSVCRT:ucrt_stubs.obj
 0001:00002cb1       ___vcrt_uninitialize       10003cb1 f   MSVCRT:ucrt_stubs.obj
 0001:00002cb1       ___vcrt_uninitialize_critical 10003cb1 f   MSVCRT:ucrt_stubs.obj
 0001:00002cb4       ___scrt_stub_for_is_c_termination_complete 10003cb4 f   MSVCRT:ucrt_stubs.obj
 0001:00002cb4       __is_c_termination_complete 10003cb4 f   MSVCRT:ucrt_stubs.obj
 0001:00002cb7       __filter_x86_sse2_floating_point_exception 10003cb7 f   MSVCRT:x86_exception_filter.obj
 0001:00002cb7       __filter_x86_sse2_floating_point_exception_default 10003cb7 f   MSVCRT:x86_exception_filter.obj
 0002:00000000       __imp__TerminateProcess@8  10004000     kernel32:KERNEL32.dll
 0002:00000004       __imp__IsDebuggerPresent@0 10004004     kernel32:KERNEL32.dll
 0002:00000008       __imp__InitializeSListHead@4 10004008     kernel32:KERNEL32.dll
 0002:0000000c       __imp__DisableThreadLibraryCalls@4 1000400c     kernel32:KERNEL32.dll
 0002:00000010       __imp__GetProcAddress@8    10004010     kernel32:KERNEL32.dll
 0002:00000014       __imp__LoadLibraryA@4      10004014     kernel32:KERNEL32.dll
 0002:00000018       __imp__SwitchToThread@0    10004018     kernel32:KERNEL32.dll
 0002:0000001c       __imp__UnhandledExceptionFilter@4 1000401c     kernel32:KERNEL32.dll
 0002:00000020       __imp__SetUnhandledExceptionFilter@4 10004020     kernel32:KERNEL32.dll
 0002:00000024       __imp__GetCurrentProcess@0 10004024     kernel32:KERNEL32.dll
 0002:00000028       __imp__GetCurrentThreadId@0 10004028     kernel32:KERNEL32.dll
 0002:0000002c       __imp__IsProcessorFeaturePresent@4 1000402c     kernel32:KERNEL32.dll
 0002:00000030       __imp__QueryPerformanceCounter@4 10004030     kernel32:KERNEL32.dll
 0002:00000034       __imp__GetCurrentProcessId@0 10004034     kernel32:KERNEL32.dll
 0002:00000038       __imp__GetSystemTimeAsFileTime@4 10004038     kernel32:KERNEL32.dll
 0002:0000003c       \177KERNEL32_NULL_THUNK_DATA 1000403c     kernel32:KERNEL32.dll
 0002:00000040       __imp____std_type_info_destroy_list 10004040     vcruntime:VCRUNTIME140.dll
 0002:00000044       __imp___except_handler4_common 10004044     vcruntime:VCRUNTIME140.dll
 0002:00000048       __imp___CxxThrowException@8 10004048     vcruntime:VCRUNTIME140.dll
 0002:0000004c       __imp____std_exception_destroy 1000404c     vcruntime:VCRUNTIME140.dll
 0002:00000050       __imp__strchr              10004050     vcruntime:VCRUNTIME140.dll
 0002:00000054       __imp____std_terminate     10004054     vcruntime:VCRUNTIME140.dll
 0002:00000058       __imp__memcmp              10004058     vcruntime:VCRUNTIME140.dll
 0002:0000005c       __imp__memset              1000405c     vcruntime:VCRUNTIME140.dll
 0002:00000060       __imp__strstr              10004060     vcruntime:VCRUNTIME140.dll
 0002:00000064       __imp____CxxFrameHandler3  10004064     vcruntime:VCRUNTIME140.dll
 0002:00000068       __imp____std_exception_copy 10004068     vcruntime:VCRUNTIME140.dll
 0002:0000006c       \177VCRUNTIME140_NULL_THUNK_DATA 1000406c     vcruntime:VCRUNTIME140.dll
 0002:00000070       __imp__free                10004070     ucrt:api-ms-win-crt-heap-l1-1-0.dll
 0002:00000074       __imp__realloc             10004074     ucrt:api-ms-win-crt-heap-l1-1-0.dll
 0002:00000078       __imp__malloc              10004078     ucrt:api-ms-win-crt-heap-l1-1-0.dll
 0002:0000007c       __imp___callnewh           1000407c     ucrt:api-ms-win-crt-heap-l1-1-0.dll
 0002:00000080       \177api-ms-win-crt-heap-l1-1-0_NULL_THUNK_DATA 10004080     ucrt:api-ms-win-crt-heap-l1-1-0.dll
 0002:00000084       __imp___execute_onexit_table 10004084     ucrt:api-ms-win-crt-runtime-l1-1-0.dll
 0002:00000088       __imp___cexit              10004088     ucrt:api-ms-win-crt-runtime-l1-1-0.dll
 0002:0000008c       __imp___initialize_onexit_table 1000408c     ucrt:api-ms-win-crt-runtime-l1-1-0.dll
 0002:00000090       __imp___initialize_narrow_environment 10004090     ucrt:api-ms-win-crt-runtime-l1-1-0.dll
 0002:00000094       __imp___configure_narrow_argv 10004094     ucrt:api-ms-win-crt-runtime-l1-1-0.dll
 0002:00000098       __imp___seh_filter_dll     10004098     ucrt:api-ms-win-crt-runtime-l1-1-0.dll
 0002:0000009c       __imp___initterm           1000409c     ucrt:api-ms-win-crt-runtime-l1-1-0.dll
 0002:000000a0       __imp___initterm_e         100040a0     ucrt:api-ms-win-crt-runtime-l1-1-0.dll
 0002:000000a4       \177api-ms-win-crt-runtime-l1-1-0_NULL_THUNK_DATA 100040a4     ucrt:api-ms-win-crt-runtime-l1-1-0.dll
 0002:000000a8       __imp____stdio_common_vsprintf 100040a8     ucrt:api-ms-win-crt-stdio-l1-1-0.dll
 0002:000000ac       __imp____stdio_common_vfprintf 100040ac     ucrt:api-ms-win-crt-stdio-l1-1-0.dll
 0002:000000b0       __imp____acrt_iob_func     100040b0     ucrt:api-ms-win-crt-stdio-l1-1-0.dll
 0002:000000b4       \177api-ms-win-crt-stdio-l1-1-0_NULL_THUNK_DATA 100040b4     ucrt:api-ms-win-crt-stdio-l1-1-0.dll
 0002:000000b8       __imp__strlen              100040b8     ucrt:api-ms-win-crt-string-l1-1-0.dll
 0002:000000bc       __imp__strcat              100040bc     ucrt:api-ms-win-crt-string-l1-1-0.dll
 0002:000000c0       __imp__strcpy              100040c0     ucrt:api-ms-win-crt-string-l1-1-0.dll
 0002:000000c4       \177api-ms-win-crt-string-l1-1-0_NULL_THUNK_DATA 100040c4     ucrt:api-ms-win-crt-string-l1-1-0.dll
 0002:000000c8       __imp__DebugCreate@8       100040c8     dbgeng:dbgeng.dll
 0002:000000cc       \177dbgeng_NULL_THUNK_DATA 100040cc     dbgeng:dbgeng.dll
 0002:000000d0       __imp__getLastErrorString@8 100040d0     java:java.dll
 0002:000000d4       __imp__JNU_NewObjectByName 100040d4     java:java.dll
 0002:000000d8       __imp__JNU_NewStringPlatform@8 100040d8     java:java.dll
 0002:000000dc       \177java_NULL_THUNK_DATA   100040dc     java:java.dll
 0002:000000e0       ___guard_check_icall_fptr  100040e0     MSVCRT:guard_support.obj
 0002:000000e4       ___castguard_check_failure_os_handled_fptr 100040e4     MSVCRT:guard_support.obj
 0002:000000e8       ___xc_a                    100040e8     MSVCRT:initializers.obj
 0002:000000ec       ___xc_z                    100040ec     MSVCRT:initializers.obj
 0002:000000f0       ___xi_a                    100040f0     MSVCRT:initializers.obj
 0002:000000f4       ___xi_z                    100040f4     MSVCRT:initializers.obj
 0002:000000f8       ___xp_a                    100040f8     MSVCRT:initializers.obj
 0002:000000fc       ___xp_z                    100040fc     MSVCRT:initializers.obj
 0002:00000100       ___xt_a                    10004100     MSVCRT:initializers.obj
 0002:00000104       ___xt_z                    10004104     MSVCRT:initializers.obj
 0002:00000108       ??_C@_0BM@DBCALOPO@decode_instructions_virtual@ 10004108     sadis.obj
 0002:00000124       ??_C@_0BG@IKDDPPGD@?$CILjava?1lang?1String?$DL?$CJV@ 10004124     sadis.obj
 0002:0000013c       ??_C@_0CL@BJCJOPKP@sun?1jvm?1hotspot?1debugger?1Debugg@ 1000413c     sadis.obj
 0002:00000168       ??_C@_0DP@IEGOKKOO@?$CILsun?1jvm?1hotspot?1asm?1Instructi@ 10004168     sadis.obj
 0002:000001a8       ??_C@_0M@IHKAILBK@handleEvent@ 100041a8     sadis.obj
 0002:000001b4       ??_C@_0DO@KENEIINN@?$CILsun?1jvm?1hotspot?1asm?1Instructi@ 100041b4     sadis.obj
 0002:000001f4       ??_C@_08DCIFBHIL@rawPrint@ 100041f4     sadis.obj
 0002:00000200       ??_C@_0BD@JFADHEFE@Ljava?1lang?1String?$DL@ 10004200     sawindbg.obj
 0002:00000214       ??_C@_09NDJHOMOJ@imagePath@ 10004214     sawindbg.obj
 0002:00000220       ??_C@_0L@IBJLJICF@symbolPath@ 10004220     sawindbg.obj
 0002:0000022c       ??_C@_01LELAEKIP@J@        1000422c     sawindbg.obj
 0002:00000230       ??_C@_0BA@ENOAPBEH@ptrIDebugClient@ 10004230     sawindbg.obj
 0002:00000240       ??_C@_0BB@FKGMCAMI@ptrIDebugControl@ 10004240     sawindbg.obj
 0002:00000254       ??_C@_0BE@HEDMCBCH@ptrIDebugDataSpaces@ 10004254     sawindbg.obj
 0002:00000268       ??_C@_0BJ@NECGJCMP@ptrIDebugOutputCallbacks@ 10004268     sawindbg.obj
 0002:00000284       ??_C@_0BC@NFADOE@ptrIDebugAdvanced@ 10004284     sawindbg.obj
 0002:00000298       ??_C@_0BB@CGICJHBO@ptrIDebugSymbols@ 10004298     sawindbg.obj
 0002:000002ac       ??_C@_0BH@MKNGBFEC@ptrIDebugSystemObjects@ 100042ac     sawindbg.obj
 0002:000002c4       ??_C@_0BI@HMPCDPNN@?$CILjava?1lang?1String?$DLJJ?$CJV@ 100042c4     sawindbg.obj
 0002:000002dc       ??_C@_0O@BAEIOKDM@addLoadObject@ 100042dc     sawindbg.obj
 0002:000002ec       ??_C@_04OHLIFDMD@?$CIJ?$CJV@ 100042ec     sawindbg.obj
 0002:000002f4       ??_C@_09IDCNHNJH@addThread@ 100042f4     sawindbg.obj
 0002:00000300       ??_C@_0ED@MJCAPJHB@?$CILjava?1lang?1String?$DLJ?$CJLsun?1jvm?1h@ 10004300     sawindbg.obj
 0002:00000344       ??_C@_0BE@PHFCBNMF@createClosestSymbol@ 10004344     sawindbg.obj
 0002:00000358       ??_C@_06FABFLPEO@?$CIJ?$FLJ?$CJV@ 10004358     sawindbg.obj
 0002:00000360       ??_C@_0BM@LHHFOJLN@setThreadIntegerRegisterSet@ 10004360     sawindbg.obj
 0002:00000380       ??_7SAOutputCallbacks@@6B@ 10004380     sawindbg.obj
 0002:00000390       __GUID_00000000_0000_0000_c000_000000000046 10004390     sawindbg.obj
 0002:000003a0       __GUID_4bf58045_d654_4c40_b0af_683090f356dc 100043a0     sawindbg.obj
 0002:000003b0       ??_C@_0CA@CHBBHPBL@out?5of?5memory?5debugger?5output?$CB?6@ 100043b0     sawindbg.obj
 0002:000003d0       __GUID_27fe5639_8407_4f47_8364_ee118fb08ac8 100043d0     sawindbg.obj
 0002:000003e0       __GUID_5182e668_105e_416e_ad92_24ef800424ba 100043e0     sawindbg.obj
 0002:000003f0       __GUID_88f7dfab_3ea7_4c3a_aefb_c4e8106173aa 100043f0     sawindbg.obj
 0002:00000400       __GUID_f2df5f53_071f_47bd_9de6_5734c3fed689 10004400     sawindbg.obj
 0002:00000410       __GUID_8c31e98c_983a_48a5_9016_6fe5d667a950 10004410     sawindbg.obj
 0002:00000420       __GUID_6b86fe2c_2c4f_4f0c_9da2_174311acc327 10004420     sawindbg.obj
 0002:00000430       ??_C@_0DG@KFKFAAAK@Windbg?5Error?3?5not?5able?5to?5creat@ 10004430     sawindbg.obj
 0002:00000468       ??_C@_0BA@IHFGPCFN@?$CFs?5?$CIhr?3?50x?$CF08X?$CJ@ 10004468     sawindbg.obj
 0002:00000478       ??_C@_0CM@HMPHNLCI@Windbg?5Error?3?5not?5able?5to?5get?5I@ 10004478     sawindbg.obj
 0002:000004a4       ??_C@_0DH@MEIJIPLO@Windbg?5Error?3?5not?5able?5to?5get?5I@ 100044a4     sawindbg.obj
 0002:000004dc       ??_C@_0DF@EJNGMFHL@Windbg?5Error?3?5not?5able?5to?5get?5I@ 100044dc     sawindbg.obj
 0002:00000514       ??_C@_0DE@BLHEEHEB@Windbg?5Error?3?5not?5able?5to?5get?5I@ 10004514     sawindbg.obj
 0002:00000548       ??_C@_0DK@CBFLKIDH@Windbg?5Error?3?5not?5able?5to?5get?5I@ 10004548     sawindbg.obj
 0002:00000584       ??_C@_0DC@OGBAOIMM@Windbg?5Error?3?5not?5able?5to?5get?5i@ 10004584     sawindbg.obj
 0002:000005b8       ??_C@_0DD@GMBHLNMH@Windbg?5Error?3?5not?5able?5to?5get?5s@ 100045b8     sawindbg.obj
 0002:000005ec       ??_C@_0CD@LLBBNFEA@Windbg?5Error?3?5OpenDumpFile?5fail@ 100045ec     sawindbg.obj
 0002:00000610       ??_C@_0CD@OHANEGIO@Windbg?5Error?3?5WaitForEvent?5fail@ 10004610     sawindbg.obj
 0002:00000634       ??_C@_0CE@NLOIALLD@Windbg?5Error?3?5AttachProcess?5fai@ 10004634     sawindbg.obj
 0002:00000658       ??_C@_0CH@OOOMOIHO@Windbg?5Error?3?5GetNumberModules?5@ 10004658     sawindbg.obj
 0002:00000680       ??_C@_0CP@GGPCODCJ@out?5of?5memory?5to?5allocate?5debug@ 10004680     sawindbg.obj
 0002:000006b0       ??_C@_0CK@OGHLJMOC@Windbg?5Error?3?5GetModuleParamete@ 100046b0     sawindbg.obj
 0002:000006dc       ??_C@_0CF@IPJIKFLG@Windbg?5Error?3?5GetModuleNames?5fa@ 100046dc     sawindbg.obj
 0002:00000704       ??_C@_0CH@DLOHNIAK@Windbg?5Error?3?5GetNumberThreads?5@ 10004704     sawindbg.obj
 0002:0000072c       ??_C@_0CG@KABLKJNP@out?5of?5memory?5to?5allocate?5threa@ 1000472c     sawindbg.obj
 0002:00000754       ??_C@_0CK@FNPIPCCJ@Windbg?5Error?3?5GetThreadIdsByInd@ 10004754     sawindbg.obj
 0002:00000780       ??_C@_0CH@DDGKENOM@Windbg?5Error?3?5SetCurrentThread?5@ 10004780     sawindbg.obj
 0002:000007a8       ??_C@_0CP@GPDFIPCF@Windbg?5Error?3?5GetCurrentThreadS@ 100047a8     sawindbg.obj
 0002:000007d8       ??_C@_0EC@GGBPHBOJ@WARNING?3?5GetThreadIdBySystemId?5@ 100047d8     sawindbg.obj
 0002:0000081c       ??_C@_0CD@EHILJEIM@Windbg?5Error?3?5CreateClient?5fail@ 1000481c     sawindbg.obj
 0002:00000840       ??_C@_0DE@HJKLOPIF@Windbg?5Error?3?5QueryInterface?5?$CII@ 10004840     sawindbg.obj
 0002:00000874       ??_C@_0CJ@LPJOGDLF@Windbg?5Error?3?5SetOutputCallback@ 10004874     sawindbg.obj
 0002:0000089d       ??_C@_00CNPNBAHC@@         1000489d     sawindbg.obj
 0002:000008a0       ??_C@_02MOLJINC@?3?3@      100048a0     sawindbg.obj
 0002:000008a8       ??_7type_info@@6B@         100048a8     MSVCRT:std_type_info_static.obj
 0002:000008ac       __pDefaultRawDllMain       100048ac     MSVCRT:dll_dllmain.obj
 0002:000008ac       __pRawDllMain              100048ac     MSVCRT:dll_dllmain.obj
 0002:000008bc       ??_7exception@std@@6B@     100048bc     MSVCRT:throw_bad_alloc.obj
 0002:000008c4       ??_C@_0BC@EOODALEL@Unknown?5exception@ 100048c4     MSVCRT:throw_bad_alloc.obj
 0002:000008dc       ??_7bad_alloc@std@@6B@     100048dc     MSVCRT:throw_bad_alloc.obj
 0002:000008e4       ??_C@_0P@GHFPNOJB@bad?5allocation@ 100048e4     MSVCRT:throw_bad_alloc.obj
 0002:000008f8       ??_7bad_array_new_length@std@@6B@ 100048f8     MSVCRT:throw_bad_alloc.obj
 0002:00000900       ??_C@_0BF@KINCDENJ@bad?5array?5new?5length@ 10004900     MSVCRT:throw_bad_alloc.obj
 0002:00000918       __load_config_used         10004918     MSVCRT:loadcfg.obj
 0002:00000a80       ??_R3IUnknown@@8           10004a80     sawindbg.obj
 0002:00000a90       ??_R2IUnknown@@8           10004a90     sawindbg.obj
 0002:00000a98       ??_R1A@?0A@EA@IUnknown@@8  10004a98     sawindbg.obj
 0002:00000ab4       ??_R3IDebugOutputCallbacks@@8 10004ab4     sawindbg.obj
 0002:00000ac4       ??_R2IDebugOutputCallbacks@@8 10004ac4     sawindbg.obj
 0002:00000ad0       ??_R1A@?0A@EA@IDebugOutputCallbacks@@8 10004ad0     sawindbg.obj
 0002:00000aec       ??_R4SAOutputCallbacks@@6B@ 10004aec     sawindbg.obj
 0002:00000b00       ??_R3SAOutputCallbacks@@8  10004b00     sawindbg.obj
 0002:00000b10       ??_R2SAOutputCallbacks@@8  10004b10     sawindbg.obj
 0002:00000b20       ??_R1A@?0A@EA@SAOutputCallbacks@@8 10004b20     sawindbg.obj
 0002:00000b3c       ??_R4type_info@@6B@        10004b3c     MSVCRT:std_type_info_static.obj
 0002:00000b50       ??_R3type_info@@8          10004b50     MSVCRT:std_type_info_static.obj
 0002:00000b60       ??_R2type_info@@8          10004b60     MSVCRT:std_type_info_static.obj
 0002:00000b68       ??_R1A@?0A@EA@type_info@@8 10004b68     MSVCRT:std_type_info_static.obj
 0002:00000b84       ??_R4exception@std@@6B@    10004b84     MSVCRT:throw_bad_alloc.obj
 0002:00000b98       ??_R3exception@std@@8      10004b98     MSVCRT:throw_bad_alloc.obj
 0002:00000ba8       ??_R2exception@std@@8      10004ba8     MSVCRT:throw_bad_alloc.obj
 0002:00000bb0       ??_R1A@?0A@EA@exception@std@@8 10004bb0     MSVCRT:throw_bad_alloc.obj
 0002:00000bcc       ??_R4bad_alloc@std@@6B@    10004bcc     MSVCRT:throw_bad_alloc.obj
 0002:00000be0       ??_R3bad_alloc@std@@8      10004be0     MSVCRT:throw_bad_alloc.obj
 0002:00000bf0       ??_R2bad_alloc@std@@8      10004bf0     MSVCRT:throw_bad_alloc.obj
 0002:00000bfc       ??_R1A@?0A@EA@bad_alloc@std@@8 10004bfc     MSVCRT:throw_bad_alloc.obj
 0002:00000c18       ??_R4bad_array_new_length@std@@6B@ 10004c18     MSVCRT:throw_bad_alloc.obj
 0002:00000c2c       ??_R3bad_array_new_length@std@@8 10004c2c     MSVCRT:throw_bad_alloc.obj
 0002:00000c3c       ??_R2bad_array_new_length@std@@8 10004c3c     MSVCRT:throw_bad_alloc.obj
 0002:00000c4c       ??_R1A@?0A@EA@bad_array_new_length@std@@8 10004c4c     MSVCRT:throw_bad_alloc.obj
 0002:00000c68       ___safe_se_handler_table   10004c68     <linker-defined>
 0002:00000c8c       ___volatile_metadata       10004c8c     <linker-defined>
 0002:00000fdc       ___rtc_iaa                 10004fdc     MSVCRT:initsect.obj
 0002:00000fe0       ___rtc_izz                 10004fe0     MSVCRT:initsect.obj
 0002:00000fe4       ___rtc_taa                 10004fe4     MSVCRT:initsect.obj
 0002:00000fe8       ___rtc_tzz                 10004fe8     MSVCRT:initsect.obj
 0002:0000127c       __TI2?AVbad_alloc@std@@    1000527c     MSVCRT:throw_bad_alloc.obj
 0002:0000128c       __CTA2?AVbad_alloc@std@@   1000528c     MSVCRT:throw_bad_alloc.obj
 0002:00001298       __CT??_R0?AVbad_alloc@std@@@8??0bad_alloc@std@@QAE@ABV01@@Z12 10005298     MSVCRT:throw_bad_alloc.obj
 0002:000012b4       __CT??_R0?AVexception@std@@@8??0exception@std@@QAE@ABV01@@Z12 100052b4     MSVCRT:throw_bad_alloc.obj
 0002:000012d0       __TI3?AVbad_array_new_length@std@@ 100052d0     MSVCRT:throw_bad_alloc.obj
 0002:000012e0       __CTA3?AVbad_array_new_length@std@@ 100052e0     MSVCRT:throw_bad_alloc.obj
 0002:000012f0       __CT??_R0?AVbad_array_new_length@std@@@8??0bad_array_new_length@std@@QAE@ABV01@@Z12 100052f0     MSVCRT:throw_bad_alloc.obj
 0002:0000170c       __IMPORT_DESCRIPTOR_dbgeng 1000570c     dbgeng:dbgeng.dll
 0002:00001720       __IMPORT_DESCRIPTOR_java   10005720     java:java.dll
 0002:00001734       __IMPORT_DESCRIPTOR_KERNEL32 10005734     kernel32:KERNEL32.dll
 0002:00001748       __IMPORT_DESCRIPTOR_VCRUNTIME140 10005748     vcruntime:VCRUNTIME140.dll
 0002:0000175c       __IMPORT_DESCRIPTOR_api-ms-win-crt-stdio-l1-1-0 1000575c     ucrt:api-ms-win-crt-stdio-l1-1-0.dll
 0002:00001770       __IMPORT_DESCRIPTOR_api-ms-win-crt-string-l1-1-0 10005770     ucrt:api-ms-win-crt-string-l1-1-0.dll
 0002:00001784       __IMPORT_DESCRIPTOR_api-ms-win-crt-heap-l1-1-0 10005784     ucrt:api-ms-win-crt-heap-l1-1-0.dll
 0002:00001798       __IMPORT_DESCRIPTOR_api-ms-win-crt-runtime-l1-1-0 10005798     ucrt:api-ms-win-crt-runtime-l1-1-0.dll
 0002:000017ac       __NULL_IMPORT_DESCRIPTOR   100057ac     dbgeng:dbgeng.dll
 0003:00000000       ___security_cookie_complement 10006000     MSVCRT:gs_cookie.obj
 0003:00000004       ___security_cookie         10006004     MSVCRT:gs_cookie.obj
 0003:00000008       ___scrt_native_dllmain_reason 10006008     MSVCRT:utility.obj
 0003:00000010       ___isa_enabled             10006010     MSVCRT:cpu_disp.obj
 0003:00000014       ___scrt_ucrt_dll_is_in_use 10006014     MSVCRT:ucrt_stubs.obj
 0003:00000018       ??_R0?AVbad_alloc@std@@@8  10006018     MSVCRT:throw_bad_alloc.obj
 0003:00000034       ??_R0?AVexception@std@@@8  10006034     MSVCRT:throw_bad_alloc.obj
 0003:00000050       ??_R0?AVbad_array_new_length@std@@@8 10006050     MSVCRT:throw_bad_alloc.obj
 0003:00000078       ??_R0?AUIUnknown@@@8       10006078     sawindbg.obj
 0003:00000090       ??_R0?AUIDebugOutputCallbacks@@@8 10006090     sawindbg.obj
 0003:000000b4       ??_R0?AVSAOutputCallbacks@@@8 100060b4     sawindbg.obj
 0003:000000d4       ??_R0?AVtype_info@@@8      100060d4     MSVCRT:std_type_info_static.obj
 0003:00000448       ?__type_info_root_node@@3U__type_info_node@@A 10006448     MSVCRT:tncleanup.obj
 0003:00000450       ?_OptionsStorage@?1??__local_stdio_scanf_options@@9@4_KA 10006450     MSVCRT:default_local_stdio_options.obj
 0003:00000458       ___scrt_current_native_startup_state 10006458     MSVCRT:utility.obj
 0003:0000045c       ___scrt_native_startup_lock 1000645c     MSVCRT:utility.obj
 0003:0000047c       ___scrt_debugger_hook_flag 1000647c     MSVCRT:utility_desktop.obj
 0003:00000480       ___isa_available           10006480     MSVCRT:cpu_disp.obj
 0003:00000484       ___favor                   10006484     MSVCRT:cpu_disp.obj
 0003:00000488       ?_OptionsStorage@?1??__local_stdio_printf_options@@9@9 10006488     <common>
 0003:00000490       ___dyn_tls_init_callback   10006490     <common>

 entry point at        0001:00002211

 Static symbols

 0000:ffff7000       .debug$S                   10000000     saproc.exp
 0000:ffff7000       .debug$S                   10000000     vcruntime:VCRUNTIME140.dll
 0000:ffff7000       .debug$S                   10000000     vcruntime:VCRUNTIME140.dll
 0000:ffff7000       .debug$S                   10000000     vcruntime:VCRUNTIME140.dll
 0000:ffff7000       .debug$S                   10000000     vcruntime:VCRUNTIME140.dll
 0000:ffff7000       .debug$S                   10000000     vcruntime:VCRUNTIME140.dll
 0000:ffff7000       .debug$S                   10000000     vcruntime:VCRUNTIME140.dll
 0000:ffff7000       .debug$S                   10000000     vcruntime:VCRUNTIME140.dll
 0000:ffff7000       .debug$S                   10000000     vcruntime:VCRUNTIME140.dll
 0000:ffff7000       .debug$S                   10000000     vcruntime:VCRUNTIME140.dll
 0000:ffff7000       .debug$S                   10000000     vcruntime:VCRUNTIME140.dll
 0000:ffff7000       .debug$S                   10000000     vcruntime:VCRUNTIME140.dll
 0000:ffff7000       .debug$S                   10000000     vcruntime:VCRUNTIME140.dll
 0000:ffff7000       .debug$S                   10000000     vcruntime:VCRUNTIME140.dll
 0000:ffff7000       .debug$S                   10000000     ucrt:api-ms-win-crt-heap-l1-1-0.dll
 0000:ffff7000       .debug$S                   10000000     ucrt:api-ms-win-crt-heap-l1-1-0.dll
 0000:ffff7000       .debug$S                   10000000     ucrt:api-ms-win-crt-heap-l1-1-0.dll
 0000:ffff7000       .debug$S                   10000000     ucrt:api-ms-win-crt-heap-l1-1-0.dll
 0000:ffff7000       .debug$S                   10000000     ucrt:api-ms-win-crt-runtime-l1-1-0.dll
 0000:ffff7000       .debug$S                   10000000     ucrt:api-ms-win-crt-runtime-l1-1-0.dll
 0000:ffff7000       .debug$S                   10000000     ucrt:api-ms-win-crt-runtime-l1-1-0.dll
 0000:ffff7000       .debug$S                   10000000     ucrt:api-ms-win-crt-runtime-l1-1-0.dll
 0000:ffff7000       .debug$S                   10000000     ucrt:api-ms-win-crt-runtime-l1-1-0.dll
 0000:ffff7000       .debug$S                   10000000     ucrt:api-ms-win-crt-runtime-l1-1-0.dll
 0000:ffff7000       .debug$S                   10000000     ucrt:api-ms-win-crt-runtime-l1-1-0.dll
 0000:ffff7000       .debug$S                   10000000     ucrt:api-ms-win-crt-runtime-l1-1-0.dll
 0000:ffff7000       .debug$S                   10000000     ucrt:api-ms-win-crt-runtime-l1-1-0.dll
 0000:ffff7000       .debug$S                   10000000     ucrt:api-ms-win-crt-runtime-l1-1-0.dll
 0000:ffff7000       .debug$S                   10000000     ucrt:api-ms-win-crt-runtime-l1-1-0.dll
 0000:ffff7000       .debug$S                   10000000     ucrt:api-ms-win-crt-runtime-l1-1-0.dll
 0000:ffff7000       .debug$S                   10000000     ucrt:api-ms-win-crt-stdio-l1-1-0.dll
 0000:ffff7000       .debug$S                   10000000     ucrt:api-ms-win-crt-stdio-l1-1-0.dll
 0000:ffff7000       .debug$S                   10000000     ucrt:api-ms-win-crt-stdio-l1-1-0.dll
 0000:ffff7000       .debug$S                   10000000     ucrt:api-ms-win-crt-string-l1-1-0.dll
 0000:ffff7000       .debug$S                   10000000     ucrt:api-ms-win-crt-string-l1-1-0.dll
 0000:ffff7000       .debug$S                   10000000     ucrt:api-ms-win-crt-string-l1-1-0.dll
 0000:ffff7000       .debug$S                   10000000     dbgeng:dbgeng.dll
 0000:ffff7000       .debug$S                   10000000     kernel32:KERNEL32.dll
 0000:ffff7000       .debug$S                   10000000     kernel32:KERNEL32.dll
 0000:ffff7000       .debug$S                   10000000     kernel32:KERNEL32.dll
 0000:ffff7000       .debug$S                   10000000     kernel32:KERNEL32.dll
 0000:ffff7000       .debug$S                   10000000     kernel32:KERNEL32.dll
 0000:ffff7000       .debug$S                   10000000     kernel32:KERNEL32.dll
 0000:ffff7000       .debug$S                   10000000     kernel32:KERNEL32.dll
 0000:ffff7000       .debug$S                   10000000     kernel32:KERNEL32.dll
 0000:ffff7000       .debug$S                   10000000     kernel32:KERNEL32.dll
 0000:ffff7000       .debug$S                   10000000     kernel32:KERNEL32.dll
 0000:ffff7000       .debug$S                   10000000     kernel32:KERNEL32.dll
 0000:ffff7000       .debug$S                   10000000     kernel32:KERNEL32.dll
 0000:ffff7000       .debug$S                   10000000     kernel32:KERNEL32.dll
 0000:ffff7000       .debug$S                   10000000     kernel32:KERNEL32.dll
 0000:ffff7000       .debug$S                   10000000     kernel32:KERNEL32.dll
 0000:ffff7000       .debug$S                   10000000     kernel32:KERNEL32.dll
 0000:ffff7000       .debug$S                   10000000     kernel32:KERNEL32.dll
 0000:ffff7000       .debug$S                   10000000     java:java.dll
 0000:ffff7000       .debug$S                   10000000     java:java.dll
 0000:ffff7000       .debug$S                   10000000     java:java.dll
 0001:00000297       _event_to_env              10001297 f   sadis.obj
 0001:000002f6       _printf_to_env             100012f6 f   sadis.obj
 0001:000003fc       ??1?$AutoArrayPtr@D@?A0x8a3339d6@@QAE@XZ 100013fc f   sawindbg.obj
 0001:000003fc       ??1?$AutoArrayPtr@K@?A0x8a3339d6@@QAE@XZ 100013fc f   sawindbg.obj
 0001:000003fc       ??1?$AutoArrayPtr@U_DEBUG_MODULE_PARAMETERS@@@?A0x8a3339d6@@QAE@XZ 100013fc f   sawindbg.obj
 0001:00000405       ??1AutoJavaByteArray@?A0x8a3339d6@@QAE@XZ 10001405 f   sawindbg.obj
 0001:00000453       ??1AutoJavaString@?A0x8a3339d6@@QAE@XZ 10001453 f   sawindbg.obj
 0001:00000612       ?WaitForEvent@@YAJPAUIDebugControl@@@Z 10001612 f   sawindbg.obj
 0001:00000650       ?addLoadObjects@@YA_NPAUJNIEnv_@@PAV_jobject@@@Z 10001650 f   sawindbg.obj
 0001:000008ea       ?addThreads@@YA_NPAUJNIEnv_@@PAV_jobject@@@Z 100018ea f   sawindbg.obj
 0001:00000dbb       ?attachToProcess@@YA_NPAUJNIEnv_@@PAV_jobject@@J@Z 10001dbb f   sawindbg.obj
 0001:00000ee3       ?getWindbgInterfaces@@YA_NPAUJNIEnv_@@PAV_jobject@@@Z 10001ee3 f   sawindbg.obj
 0001:000011af       ?openDumpFile@@YA_NPAUJNIEnv_@@PAV_jobject@@PAV_jstring@@@Z 100021af f   sawindbg.obj
 0001:000012f2       ?releaseWindbgInterfaces@@YA_NPAUJNIEnv_@@PAV_jobject@@@Z 100022f2 f   sawindbg.obj
 0001:00001421       ?setImageAndSymbolPath@@YA_NPAUJNIEnv_@@PAV_jobject@@@Z 10002421 f   sawindbg.obj
 0001:00001541       ?throwNewDebuggerException@@YAXPAUJNIEnv_@@PBD@Z 10002541 f   sawindbg.obj
 0001:00001df0       $$000000                   10002df0     MSVCRT:chkstk.obj
 0001:00001e04       cs10                       10002e04     MSVCRT:chkstk.obj
 0001:00001e12       cs20                       10002e12     MSVCRT:chkstk.obj
 0001:00001ed1       ?dllmain_crt_dispatch@@YGHQAUHINSTANCE__@@KQAX@Z 10002ed1 f   MSVCRT:dll_dllmain.obj
 0001:00001f24       ?dllmain_crt_process_attach@@YAHQAUHINSTANCE__@@QAX@Z 10002f24 f   MSVCRT:dll_dllmain.obj
 0001:0000202b       ?dllmain_crt_process_detach@@YAH_N@Z 1000302b f   MSVCRT:dll_dllmain.obj
 0001:000020db       ?dllmain_dispatch@@YAHQAUHINSTANCE__@@KQAX@Z 100030db f   MSVCRT:dll_dllmain.obj
 0001:000021e6       ?dllmain_raw@@YGHQAUHINSTANCE__@@KQAX@Z 100031e6 f   MSVCRT:dll_dllmain.obj
 0001:00002472       ___get_entropy             10003472 f   MSVCRT:gs_support.obj
 0001:00002567       ?find_pe_section@@YAPAU_IMAGE_SECTION_HEADER@@QAEI@Z 10003567 f   MSVCRT:utility.obj
 0001:000029c0       $$000000                   100039c0     MSVCRT:sehprolg4.obj
 0001:00002d2f       __ehhandler$??1AutoJavaByteArray@?A0x8a3339d6@@QAE@XZ 10003d2f f   sawindbg.obj
 0001:00002d2f       __ehhandler$??1AutoJavaString@?A0x8a3339d6@@QAE@XZ 10003d2f f   sawindbg.obj
 0001:00002d4c       __unwindfunclet$?addLoadObjects@@YA_NPAUJNIEnv_@@PAV_jobject@@@Z$0 10003d4c f   sawindbg.obj
 0001:00002d54       __unwindfunclet$?addLoadObjects@@YA_NPAUJNIEnv_@@PAV_jobject@@@Z$1 10003d54 f   sawindbg.obj
 0001:00002d5c       __unwindfunclet$?addLoadObjects@@YA_NPAUJNIEnv_@@PAV_jobject@@@Z$2 10003d5c f   sawindbg.obj
 0001:00002d64       __unwindfunclet$?addLoadObjects@@YA_NPAUJNIEnv_@@PAV_jobject@@@Z$3 10003d64 f   sawindbg.obj
 0001:00002d71       __ehhandler$?addLoadObjects@@YA_NPAUJNIEnv_@@PAV_jobject@@@Z 10003d71 f   sawindbg.obj
 0001:00002d9b       __unwindfunclet$?addThreads@@YA_NPAUJNIEnv_@@PAV_jobject@@@Z$0 10003d9b f   sawindbg.obj
 0001:00002da3       __unwindfunclet$?addThreads@@YA_NPAUJNIEnv_@@PAV_jobject@@@Z$1 10003da3 f   sawindbg.obj
 0001:00002dab       __unwindfunclet$?addThreads@@YA_NPAUJNIEnv_@@PAV_jobject@@@Z$2 10003dab f   sawindbg.obj
 0001:00002db3       __unwindfunclet$?addThreads@@YA_NPAUJNIEnv_@@PAV_jobject@@@Z$3 10003db3 f   sawindbg.obj
 0001:00002dbb       __unwindfunclet$?addThreads@@YA_NPAUJNIEnv_@@PAV_jobject@@@Z$5 10003dbb f   sawindbg.obj
 0001:00002dc3       __unwindfunclet$?addThreads@@YA_NPAUJNIEnv_@@PAV_jobject@@@Z$4 10003dc3 f   sawindbg.obj
 0001:00002dd0       __ehhandler$?addThreads@@YA_NPAUJNIEnv_@@PAV_jobject@@@Z 10003dd0 f   sawindbg.obj
 0001:00002dfa       __unwindfunclet$?attachToProcess@@YA_NPAUJNIEnv_@@PAV_jobject@@J@Z$0 10003dfa f   sawindbg.obj
 0001:00002e02       __unwindfunclet$?attachToProcess@@YA_NPAUJNIEnv_@@PAV_jobject@@J@Z$1 10003e02 f   sawindbg.obj
 0001:00002e0f       __ehhandler$?attachToProcess@@YA_NPAUJNIEnv_@@PAV_jobject@@J@Z 10003e0f f   sawindbg.obj
 0001:00002e2c       __unwindfunclet$?getWindbgInterfaces@@YA_NPAUJNIEnv_@@PAV_jobject@@@Z$0 10003e2c f   sawindbg.obj
 0001:00002e34       __unwindfunclet$?getWindbgInterfaces@@YA_NPAUJNIEnv_@@PAV_jobject@@@Z$1 10003e34 f   sawindbg.obj
 0001:00002e3c       __unwindfunclet$?getWindbgInterfaces@@YA_NPAUJNIEnv_@@PAV_jobject@@@Z$2 10003e3c f   sawindbg.obj
 0001:00002e44       __unwindfunclet$?getWindbgInterfaces@@YA_NPAUJNIEnv_@@PAV_jobject@@@Z$4 10003e44 f   sawindbg.obj
 0001:00002e4c       __unwindfunclet$?getWindbgInterfaces@@YA_NPAUJNIEnv_@@PAV_jobject@@@Z$5 10003e4c f   sawindbg.obj
 0001:00002e54       __unwindfunclet$?getWindbgInterfaces@@YA_NPAUJNIEnv_@@PAV_jobject@@@Z$6 10003e54 f   sawindbg.obj
 0001:00002e61       __ehhandler$?getWindbgInterfaces@@YA_NPAUJNIEnv_@@PAV_jobject@@@Z 10003e61 f   sawindbg.obj
 0001:00002e7e       __unwindfunclet$?openDumpFile@@YA_NPAUJNIEnv_@@PAV_jobject@@PAV_jstring@@@Z$0 10003e7e f   sawindbg.obj
 0001:00002e86       __unwindfunclet$?openDumpFile@@YA_NPAUJNIEnv_@@PAV_jobject@@PAV_jstring@@@Z$1 10003e86 f   sawindbg.obj
 0001:00002e8e       __unwindfunclet$?openDumpFile@@YA_NPAUJNIEnv_@@PAV_jobject@@PAV_jstring@@@Z$2 10003e8e f   sawindbg.obj
 0001:00002e9b       __ehhandler$?openDumpFile@@YA_NPAUJNIEnv_@@PAV_jobject@@PAV_jstring@@@Z 10003e9b f   sawindbg.obj
 0001:00002eb8       __unwindfunclet$?setImageAndSymbolPath@@YA_NPAUJNIEnv_@@PAV_jobject@@@Z$0 10003eb8 f   sawindbg.obj
 0001:00002ec0       __unwindfunclet$?setImageAndSymbolPath@@YA_NPAUJNIEnv_@@PAV_jobject@@@Z$1 10003ec0 f   sawindbg.obj
 0001:00002ecd       __ehhandler$?setImageAndSymbolPath@@YA_NPAUJNIEnv_@@PAV_jobject@@@Z 10003ecd f   sawindbg.obj
 0001:00002eea       __ehhandler$_Java_sun_jvm_hotspot_debugger_windbg_WindbgDebuggerLocal_consoleExecuteCommand0@12 10003eea f   sawindbg.obj
 0002:000008b0       _GS_ExceptionPointers      100048b0     MSVCRT:gs_report.obj
 0002:00000ff0       __ehfuncinfo$_Java_sun_jvm_hotspot_debugger_windbg_WindbgDebuggerLocal_consoleExecuteCommand0@12 10004ff0     sawindbg.obj
 0002:00001014       __unwindtable$_Java_sun_jvm_hotspot_debugger_windbg_WindbgDebuggerLocal_consoleExecuteCommand0@12 10005014     sawindbg.obj
 0002:00001064       __ehfuncinfo$??1AutoJavaByteArray@?A0x8a3339d6@@QAE@XZ 10005064     sawindbg.obj
 0002:00001064       __ehfuncinfo$??1AutoJavaString@?A0x8a3339d6@@QAE@XZ 10005064     sawindbg.obj
 0002:00001088       __ehfuncinfo$?getWindbgInterfaces@@YA_NPAUJNIEnv_@@PAV_jobject@@@Z 10005088     sawindbg.obj
 0002:000010ac       __unwindtable$?getWindbgInterfaces@@YA_NPAUJNIEnv_@@PAV_jobject@@@Z 100050ac     sawindbg.obj
 0002:000010dc       __unwindtable$?setImageAndSymbolPath@@YA_NPAUJNIEnv_@@PAV_jobject@@@Z 100050dc     sawindbg.obj
 0002:000010ec       __ehfuncinfo$?setImageAndSymbolPath@@YA_NPAUJNIEnv_@@PAV_jobject@@@Z 100050ec     sawindbg.obj
 0002:00001110       __unwindtable$?openDumpFile@@YA_NPAUJNIEnv_@@PAV_jobject@@PAV_jstring@@@Z 10005110     sawindbg.obj
 0002:00001128       __ehfuncinfo$?openDumpFile@@YA_NPAUJNIEnv_@@PAV_jobject@@PAV_jstring@@@Z 10005128     sawindbg.obj
 0002:0000114c       __unwindtable$?attachToProcess@@YA_NPAUJNIEnv_@@PAV_jobject@@J@Z 1000514c     sawindbg.obj
 0002:0000115c       __ehfuncinfo$?attachToProcess@@YA_NPAUJNIEnv_@@PAV_jobject@@J@Z 1000515c     sawindbg.obj
 0002:00001180       __unwindtable$?addLoadObjects@@YA_NPAUJNIEnv_@@PAV_jobject@@@Z 10005180     sawindbg.obj
 0002:000011a0       __ehfuncinfo$?addLoadObjects@@YA_NPAUJNIEnv_@@PAV_jobject@@@Z 100051a0     sawindbg.obj
 0002:000011c4       __ehfuncinfo$?addThreads@@YA_NPAUJNIEnv_@@PAV_jobject@@@Z 100051c4     sawindbg.obj
 0002:000011e8       __unwindtable$?addThreads@@YA_NPAUJNIEnv_@@PAV_jobject@@@Z 100051e8     sawindbg.obj
 0002:00001218       __sehtable$?dllmain_crt_process_attach@@YAHQAUHINSTANCE__@@QAX@Z 10005218     MSVCRT:dll_dllmain.obj
 0002:00001238       __sehtable$?dllmain_crt_process_detach@@YAH_N@Z 10005238     MSVCRT:dll_dllmain.obj
 0002:00001260       __sehtable$?dllmain_dispatch@@YAHQAUHINSTANCE__@@KQAX@Z 10005260     MSVCRT:dll_dllmain.obj
 0002:00001310       __sehtable$___scrt_is_nonwritable_in_current_image 10005310     MSVCRT:utility.obj
 0002:00001330       .edata                     10005330     saproc.exp
 0002:00001358       rgpv                       10005358     saproc.exp
 0002:00001384       rgszName                   10005384     saproc.exp
 0002:000013b0       rgwOrd                     100053b0     saproc.exp
 0002:000013c6       szName                     100053c6     saproc.exp
 0002:000013d1       $N00001                    100053d1     saproc.exp
 0002:00001402       $N00002                    10005402     saproc.exp
 0002:0000143a       $N00003                    1000543a     saproc.exp
 0002:00001482       $N00004                    10005482     saproc.exp
 0002:000014ef       $N00005                    100054ef     saproc.exp
 0002:00001543       $N00006                    10005543     saproc.exp
 0002:00001587       $N00007                    10005587     saproc.exp
 0002:000015da       $N00008                    100055da     saproc.exp
 0002:0000161e       $N00009                    1000561e     saproc.exp
 0002:0000166c       $N00010                    1000566c     saproc.exp
 0002:000016b7       $N00011                    100056b7     saproc.exp
 0002:000018ae       .idata$6                   100058ae     dbgeng:dbgeng.dll
 0002:00001904       .idata$6                   10005904     java:java.dll
 0002:00001a66       .idata$6                   10005a66     kernel32:KERNEL32.dll
 0002:00001b46       .idata$6                   10005b46     vcruntime:VCRUNTIME140.dll
 0002:00001c8a       .idata$6                   10005c8a     ucrt:api-ms-win-crt-stdio-l1-1-0.dll
 0002:00001caa       .idata$6                   10005caa     ucrt:api-ms-win-crt-string-l1-1-0.dll
 0002:00001ccc       .idata$6                   10005ccc     ucrt:api-ms-win-crt-heap-l1-1-0.dll
 0002:00001cec       .idata$6                   10005cec     ucrt:api-ms-win-crt-runtime-l1-1-0.dll
 0003:000000f0       ?imagePath_ID@@3PAU_jfieldID@@A 100060f0     sawindbg.obj
 0003:000000f4       ?symbolPath_ID@@3PAU_jfieldID@@A 100060f4     sawindbg.obj
 0003:000000f8       ?ptrIDebugClient_ID@@3PAU_jfieldID@@A 100060f8     sawindbg.obj
 0003:000000fc       ?ptrIDebugControl_ID@@3PAU_jfieldID@@A 100060fc     sawindbg.obj
 0003:00000100       ?ptrIDebugDataSpaces_ID@@3PAU_jfieldID@@A 10006100     sawindbg.obj
 0003:00000104       ?ptrIDebugOutputCallbacks_ID@@3PAU_jfieldID@@A 10006104     sawindbg.obj
 0003:00000108       ?ptrIDebugAdvanced_ID@@3PAU_jfieldID@@A 10006108     sawindbg.obj
 0003:0000010c       ?ptrIDebugSymbols_ID@@3PAU_jfieldID@@A 1000610c     sawindbg.obj
 0003:00000110       ?ptrIDebugSystemObjects_ID@@3PAU_jfieldID@@A 10006110     sawindbg.obj
 0003:00000114       ?addLoadObject_ID@@3PAU_jmethodID@@A 10006114     sawindbg.obj
 0003:00000118       ?addThread_ID@@3PAU_jmethodID@@A 10006118     sawindbg.obj
 0003:0000011c       ?createClosestSymbol_ID@@3PAU_jmethodID@@A 1000611c     sawindbg.obj
 0003:00000120       ?setThreadIntegerRegisterSet_ID@@3PAU_jmethodID@@A 10006120     sawindbg.obj
 0003:00000124       ?__proc_attached@@3HA      10006124     MSVCRT:dll_dllmain.obj
 0003:00000128       _GS_ExceptionRecord        10006128     MSVCRT:gs_report.obj
 0003:00000178       _GS_ContextRecord          10006178     MSVCRT:gs_report.obj
 0003:00000460       ?is_initialized_as_dll@@3_NA 10006460     MSVCRT:utility.obj
 0003:00000461       ?module_local_atexit_table_initialized@@3_NA 10006461     MSVCRT:utility.obj
 0003:00000464       ?module_local_atexit_table@@3U_onexit_table_t@@A 10006464     MSVCRT:utility.obj
 0003:00000470       ?module_local_at_quick_exit_table@@3U_onexit_table_t@@A 10006470     MSVCRT:utility.obj
 0004:00000060       $R000000                   10007060     saproc.dll.res
